:1000000012C02CC02BC02AC029C029C027C026C0BE
:1000100093C024C023C022C021C020C01FC01EC066
:100020001DC01CC01BC011241FBECFE5D4E0DEBF25
:10003000CDBF13E0A0E6B0E0EEEDF4E002C0059025
:100040000D92A439B107D9F713E0A4E9B3E001C0D8
:100050001D92AF39B107E1F794D03FC2D1CF1F92C3
:100060000F920FB60F9211242F933F934F935F93EC
:100070006F937F938F939F93AF93BF93EF93FF9370
:100080002CB53DB58091940390919503A091960372
:10009000B0919703DC019927882740E050E0820F58
:1000A000931FA41FB51F77E0B695A79597958795E1
:1000B0007A95D1F78093980390939903A0939A032C
:1000C000B0939B038CB59DB520919403309195031B
:1000D0004091960350919703A90133272227A0E06E
:1000E000B0E0280F391F4A1F5B1F60E078E38CE9FE
:1000F0009CE1BDD130939E0320939D031DBC1CBC8D
:100100001092940310929503109296031092970305
:1001100081E080939C03FF91EF91BF91AF919F91FC
:100120008F917F916F915F914F913F912F910F90A0
:100130000FBE0F901F9018951F920F920FB60F923F
:1001400011248F939F93AF93BF93809194039091C9
:100150009503A0919603B09197030196A11DB11D3F
:100160008093940390939503A0939603B093970381
:10017000BF91AF919F918F910F900FBE0F901F90E5
:1001800018953F924F925F926F927F928F929F92BB
:10019000AF92BF92CF92DF92EF92FF920F931F9395
:1001A000DF93CF93CDB7DEB72D970FB6F894DEBFB0
:1001B0000FBECDBF81E48EBD84E289BF17BA8FEF39
:1001C00081BB82BB7894FE0131968BE0DF011D92EA
:1001D0008A95E9F760E07724AA24BB2465014424CA
:1001E000552434EF832E31E0932E3E2E6F2EFE01E8
:1001F0003796FD87EC8780919C03813009F09AC087
:1002000010929C030894411C511CF1E24F16F3E03C
:100210005F063CF0739485E0871508F47724442446
:100220005524A0909803B0909903C0909A03D09061
:100230009B0395E0791609F070C0A5E18A16910438
:100240000CF465C080919D0390919E034AE050E0BC
:10025000632D762DDDD0832D962D8C0140E050E06E
:1002600065E070E0F8019081892F80538A30C8F0F2
:10027000FA01EF51FD4F1082FA01EE51FD4F10824D
:10028000FA01ED51FD4F1082FA01EC51FD4F108241
:10029000FA01EB51FD4F1082FB01EF51FD4F10822F
:1002A00027C0892F90E0C097DC01AA0FBB1FAA0FBF
:1002B000BB1FA80FB91FAF59BC4F20E030E091EE33
:1002C000E92E92E0F92EE60EF71E2530310519F4DD
:1002D000F701108207C0F901E40FF51F8C91EF516F
:1002E000FD4F80832F5F3F4F11962630310569F710
:1002F0000F5F1F4F4A5F5F4F6A5F7F4F8C859D8501
:100300000817190709F0AECF8824992403C0089470
:10031000811C911C8091E1020AC0E72DF0E0F69566
:10032000FE2FEE27F795E795E05AFF4F808182BBBD
:1003300060E061CF2CB53DB5809194039091950319
:10034000A0919603B0919703DC019927882740E09C
:1003500050E0820F931FA41FB51FA816B906CA0646
:10036000DB0630F56F5F67FD6FE7A62FB0E095E025
:10037000791669F0E72DF0E0F695FE2FEE27F79558
:10038000E795EA0FFB1FE05AFF4F808103C0AF5192
:10039000BD4F8C9182BB8091980390919903A0915D
:1003A0009A03B0919B03A80EB91ECA1EDB1E23CF71
:1003B0008CB59DB52091940330919503409196039F
:1003C00050919703E0909803F090990300919A035D
:1003D00010919B03A90133272227A0E0B0E0280F4A
:1003E000391F4A1F5B1FF2E016950795F794E794B3
:1003F000FA95D1F7D601C5018E199F09A00BB10B53
:1004000082179307A407B50708F0F5CE12BAF3CE0A
:10041000FB019F01E8944230BCF04532ACF44A3015
:1004200029F497FB1EF4909581959F4F642F7727B1
:1004300040D0805D8A330CF0895D8193CB010097B9
:10044000A9F716F45DE251931082C90100C0DC01E6
:10045000FC01672F71917723E1F7329704C07C91FB
:100460006D9370836291AE17BF07C8F30895A1E240
:100470001A2EAA1BBB1BFD010DC0AA1FBB1FEE1F1E
:10048000FF1FA217B307E407F50720F0A21BB30B69
:10049000E40BF50B661F771F881F991F1A9469F7E5
:1004A00060957095809590959B01AC01BD01CF0141
:1004B0000895AA1BBB1B51E107C0AA1FBB1FA617AB
:1004C000B70710F0A61BB70B881F991F5A95A9F7FD
:0E04D00080959095BC01CD010895F894FFCF62
:1004DE00C0C0C0E0E0F0F0F8F8FCFCFCFEFEFEFF51
:1004EE00FFFFFFFFFFFFFFFFFFFFFFFFFFFFFEFE10
:1004FE00FEFCFCF8F8F8F0F0F0F0E0E0E0E0E0E010
:10050E00E0E0E0E0E0E0E0E0E0E0E0E0F0F0F0F09D
:10051E00F8F0F0F0F0E0E0E0E0E0E0E0E0E0E0E075
:10052E00E0E0E0E0E0E0E0F0F0F0F0F8F8F8FCFCFD
:10053E00FEFEFEFEFFFFFFFFFFFFFFFFFFFFFFFFC1
:10054E00FFFFFEFEFEFCFCFCF8F8F0F0E0E0C0C0A1
:10055E0001010101010131797979797979F1F1F1AD
:10056E00616141010101010101010101010101016D
:10057E00010101010121213119191919111119193D
:10058E0019191919191919191919191919191919CD
:10059E0019191919191919191919191919191919BD
:1005AE001911111111191919193121210101010105
:1005BE00010101010101010101010101010141617D
:1005CE0061F1F1F1797979797979310101010101DD
:1005DE00FFFFFFFFFFFFFFFFFFFFFFFFC101010155
:1005EE00010101010101010101010101010101FFEF
:1005FE00FFFFFFFFFFFFFFFFFFFFFFFFFFFFFFFFFD
:10060E00FFFF7F3F01010101010101010101010114
:10061E0001010101010101010101FFFFFFFFFFFFC8
:10062E00FFFFFFFFFFFFFFFFFFFFFFFFFFFFFFFFCC
:10063E00FFFF0101010101010101010101010101A0
:10064E00010101010101031F7FFFFFFFFFFFFFFFFC
:10065E00F1F1F9F9E1C1C18181818185858D8D9D90
:10066E00BDFDFDFDFDFDFDFDFDFDFDFDFDFDFDFDEC
:10067E00FDFDFDFDFDFDFDFDFDFDFDDDCDCDCDCD7C
:10068E00C1C181818081C1E1F1E1C181808181C1DE
:10069E00C1CDCDCDCDDDFDFDFDFDFDFDFDFDFDFD98
:1006AE00FDFDFDFDFDFDFDFDFDFDFDFDFDFDFDFD6C
:1006BE00BD9D8D8D858581818181C1C1E1F9F9F164
:1006CE00414101010101010101010101010101018C
:1006DE00FFFCF8F0E0E0C0C08080808000000000E9
:1006EE000080808080C0C0E0F0F8FCFFFEFCF8F0D7
:1006FE00F0E0E0E0C0C0C0C08080808080C0C0E07C
:10070E00E0F0F8FEFFFFFEFCF8F8F0F0E0E0E0C0ED
:10071E00C0C0E0E0E0F0F0F8FCFEFFFFFEFCF8F0F9
:10072E00E0E0C0C0C0808080C0C0C0C0C0E0E0E0DB
:10073E00F0F8F8FCFEFFFCF0E0E0C0C080808080A6
:10074E000000000080808080C0C0C0E0E0F0F8FCB7
:10075E000500000000000000000000000000000086
:10076E00000000000000000000000000000000007B
:10077E00000000000000000000000000000000006B
:10078E00000000000000000000003E414141220038
:10079E003C4040207C007C08040408007C080404D3
:1007AE0008003854545418007C0804047800043FA0
:1007BE00444020000000000000007F091929460077
:1007CE007F09090906007F020C027F000036360001
:1007DE00003E5149453E00427F400042615149462C
:1007EE002141454B311814127F1027454545393CA0
:1007FE004A494930030171090736494949360649C4
:04080E0049291E0056
:00000001FF
